:020000040000FA
:020000001228C4
:08000800BA00030E8301BB00E6
:100010000A08BC003C088A003B0E8300BA0E3A0E68
:100020000C1009008316FF30850000308600013077
:100030008700811384309F008312C6308700D70168
:10004000D601EB01EC018A1562268A112A24861753
:10005000851A2F28F22312245714851E2D28051ADD
:100060003628F2231224D717051E342805193B28F9
:10007000F2231224532604305124EA000030512484
:10008000E90002305124E80014305124E00010301F
:100090005124DF000C305124DE0057185428D71BA0
:1000A0005428051A5528561456285610D71B2025B3
:1000B000571875245618FE25EC0F6328EB0A0330F9
:1000C0006B020319861312241224122456186D2869
:1000D00057186D28D71B6D28051970288A15002818
:1000E000D63087008316213087008312042486309F
:1000F00087006923D63087003E08DA003D08DB0020
:1001000003305A0203198A288316013087008312AC
:100110001224C62859245A08A1005B08A000073001
:10012000A4006524692445244D24452452303D24EF
:1001300078303D243E303D243408303E3D2435089F
:10014000303E3D243608303E3D2401303D242030F1
:100150003D243D303D2453303D2463303D24613007
:100160003D246E303D243D303D2449244D24492416
:1001700043303D2478303D243E303D242D303D2415
:100180002D303D242D303D2479234D28EB01EC0109
:10019000D63087000424463087006923D630870094
:1001A0003E08D8003D08D9000424463087000630B8
:1001B000BE00BE0BD92800006923D63087003E0858
:1001C000DA003D08DB0003305A0203192B295924B9
:1001D0005A08A1005B08A0005808A5005908A4000F
:1001E0006124A308031D59245D242108A5002008CB
:1001F000A4005808A1005908A0006124A308031D09
:1002000059245D2408305124A4006124A308031D4F
:1002100059242108D3002008D20059240330A50016
:100220006930A4005E08A00071245D245308A50075
:100230005208A4006D245D240130A5005530A400AF
:1002400065242108DC002008DD005717D71257125B
:1002500056184D28402A831621308700831209241E
:10026000463087006923D63087003E08D8003D0815
:10027000D9000424463087000630BE00BE0B3E295C
:1002800000006923D63087003E08DA003D08DB0015
:10029000831601308700831203305A020319842920
:1002A00059245A08A1005B08A0005808A500590865
:1002B000A4006124A308031D59245D246630A40012
:1002C0006D242108D3002008D20059245808A10029
:1002D0005908A0005F08A4006D245D245308A50000
:1002E0005208A4006124A308031D59245D2425306D
:1002F000A40065242108DC002008DD005713D71670
:10030000571256184D28F029831621308700831282
:100310000424863087006923D63087003E08D80041
:100320003D08D9000424863087000230BE00BE0B91
:100330009729000000006923D63087003E08DA00C4
:100340003D08DB00831601308700831203305A0218
:100350000319DE2959245A08A1005B08A000580897
:10036000A5005908A4006124A308031D59245D2495
:10037000D230A4006D242108D3002008D2005924D3
:100380005808A1005908A0006008A4006D245D244D
:100390005308A5005208A4006124A308031D592492
:1003A0005D244730A40065242108DC002008DD001E
:1003B0005713D712571656184D281B2A45244D247B
:1003C000452445303D2473303D2472303D243E3079
:1003D0003D242D303D242D303D242D303D241B2A3D
:1003E00059245A08A1005B08A0005808A500590824
:1003F000A40061242108D3002008D2005D243230FB
:10040000A4006124A308031D402A59240430A1003C
:100410006030A0006908A40071245D243630A40077
:100420006D245D245308A5005208A4006524D7104C
:100430005715D711E72A59245A08A1005B08A000D4
:100440005808A5005908A40061242108D3002008F9
:10045000D2005D240530A4006124A308031DC92A2D
:1004600059243230A0006A08A4006D245D2453088A
:10047000A5005208A4006524D7105711D715E72A04
:100480001430E7000130E500E601831621308700D3
:10049000831204244630870069233E08E1003D08AA
:1004A000E20000005A2A00000000000000000000E6
:1004B000000000000000000000000000000000003C
:1004C000000000000000000000000000000000002C
:1004D000692302303E0203187E2AE50F532AE60AFA
:1004E0003E086102031D592A62083D02BF00023026
:1004F0003F02031CC92AE70B612AC92AD6308700AC
:100500003E08E3003D08E4008316013087008312B3
:1005100059240A30A0006808A4006D245D2410301E
:10052000A500DE30A40071245D246508A4006608DF
:10053000A5006D242308D5002208D4002108D3008B
:100540002008D20059246308A1006408A0006108B3
:10055000A5006208A40061242108BE002008BD0097
:100560005D240530A4006124A308031DC92A592471
:100570003E08A5003D08A4005508A3005408A200A9
:100580005308A1005208A0006524D7145711D711B1
:10059000E72AD6308700831601308700831249246A
:1005A0004D24492443303D2478303D243E303D24C1
:1005B0002D303D242D303D246E303D246F303D24C0
:1005C0002D303D242D303D24561BC923352B692465
:1005D00049244D24492443303D2478303D243E3085
:1005E0003D24D71C1D2B013032020318002B013093
:1005F00033020318032B013034020318082B0E2B8F
:100600003208303E3D243308303E3D2420303D2426
:100610003408303E3D24B208031D182B3508303E07
:100620003D24B308031D1A2B3608303E3D241C2BF5
:1006300030303D2430303D24312BB3080319232BB7
:100640003308303E3D243408303E3D242E303D24D6
:100650003508303E3D24B308031D312B3608303EAB
:100660003D2402303D2446303D2459245C08A1003D
:100670005D08A000692445244D24452452303D24C2
:1006800078303D243E303D24571B492BB3080319D5
:100690004C2B3308303E3D24571F502B2C303D242B
:1006A0003408303E3D24D71E572B2C303D243508CE
:1006B000303E3D24571E5E2B2C303D24D71E632B2D
:1006C000B308031D662B3608303E3D2401303D241F
:1006D0004D2881309F000530BE00BE0B6D2B1F15CD
:1006E0001F19702B1E08BE0083161E088312BD0042
:1006F0000800592489309F000530BE00BE0B7E2BB8
:100700001F151F19812B1E08D30083161E08831284
:10071000D2005308A1005208A000CE30412402307C
:100720002102031D962B03303D24C82B5924530866
:10073000A1005208A0000130A500E330A40061240C
:10074000A308031DA62B04303D24C82B59245308AD
:10075000A1005208A0000130A500C730A400612408
:10076000A308031DB62B05303D24C82B592453087C
:10077000A1005208A0000130A500AB30A400612404
:10078000A308031DC62B06303D24C82B07303D248B
:10079000080059245808A1005908A0000830512425
:1007A000A4006124A308031D59242108D3002008B4
:1007B000D20059240330A5006930A4005E08A000CF
:1007C00071245D245308A5005208A4006D245D2403
:1007D0000130A5005530A40065242108DC00200864
:1007E000DD000800452420303D2453303D24653091
:1007F0003D2472303D2476303D2469303D24633001
:100800003D2465303D240800FF30BE00BE0B062CA1
:100810000800ED30BE004130BF00BE0B0D2CBF0BF9
:100820000D2C0800DC30BE008230BF00BE0B162C41
:10083000BF0B162C00000800AC30BE001330BF0008
:100840000630C000BE0B222CBF0B222CC00B222C6A
:100850000000080048308A159B268A1107308A005C
:100860003830C2000030C30000278A1580268A1164
:10087000C30A4308C20B342C08008A1580268A114B
:1008800008008A159B268A1108008A15B2268A114B
:1008900008008A15B7268A1108008A15C1268A1110
:1008A00008008A155F248A1108008A156A248A11B3
:1008B00008008A1509258A1108008A1504258A115D
:1008C00008008A1516258A1108008A153A258A110A
:1008D00008008A15CB258A1108008A1523258A115C
:1008E00008008A1519258A110800D7197B2C571979
:1008F000B22CD718E92C051A7E2CEA0A851A812C0D
:10090000EA0345244D246A08A0007F30A400612436
:100910006924452420303D2431303D2475303D2468
:100920003E303D242C1C962C2D303D243408303E86
:100930003D243508303E3D243608303E3D243C30D1
:100940003D2420303D240519B12C45244D24452457
:100950008A15C6248A116A08BD0004305524051D75
:10096000AF2C0800051AB52CE90A851AB82CE90342
:1009700045244D246908A0007F30A4006124692427
:10098000452420303D2439303D2475303D243E300F
:100990003D242C1CCD2C2D303D243408303E3D24EC
:1009A0003508303E3D243608303E3D243C303D2461
:1009B00020303D240519E82C45244D2445248A1572
:1009C000C6248A116908BD0000305524051DE62C97
:1009D0000800051AEC2CE80A851AEF2CE8034524D8
:1009E0004D246808A0007F30A400612469244524B8
:1009F00020303D2439303D2475303D243E303D24A7
:100A00002C1C042D2D303D243408303E3D24350867
:100A1000303E3D243608303E3D243C303D242030DD
:100A20003D2405191F2D45244D2445248A15C6242F
:100A30008A116808BD0002305524051D1D2D0800CF
:100A4000571B262DD71A5E2D571A962D051A292DBC
:100A5000DE0A851A2C2DDE0345244D245E08A000F5
:100A60007F30A40061246924452420303D243130A6
:100A70003D2452303D243E303D242C1C412D2D3050
:100A80003D243408303E3D243508303E3D243608B0
:100A9000303E3D243C303D2420303D2405195C2D62
:100AA00045244D2445248A15C6248A115E08BD00BC
:100AB0000C305524051D5A2DCE250800051A612D30
:100AC000DF0A851A642DDF0345244D245F08A0004A
:100AD0006430A40061246924452420303D24313051
:100AE0003D2430303D2452303D242C1C792D2D30B6
:100AF0003D243408303E3D243508303E3D24360840
:100B0000303E3D243C303D2420303D240519942DB9
:100B100045244D2445248A15C6248A115F08BD004A
:100B200010305524051D922DCE250800051A992D4B
:100B3000E00A851A9C2DE00345244D246008A0009E
:100B40006430A40061246924452420303D243430DD
:100B50003D2430303D2452303D242C1CB12D2D300D
:100B60003D243408303E3D243508303E3D243608CF
:100B7000303E3D243C303D2420303D240519CC2D11
:100B800045244D2445248A15C6248A116008BD00D9
:100B900014305524051DCA2DCE25080059245C08A3
:100BA000A1005D08A000692449244D244924203077
:100BB0003D24571BDE2DB3080319E12D3308303EC9
:100BC0003D24571FE52D2C303D243408303E3D2474
:100BD000D71EEC2D2C303D243508303E3D24571EC9
:100BE000F32D2C303D24D71EF82DB308031DFB2D0B
:100BF0003608303E3D2401303D2408005808A1004D
:100C00005908A000692445244D24452420303D2462
:100C10003408303E3D243508303E3D243608303E11
:100C20003D24571F152E2B303D24D71E192E2F3053
:100C30003D24571E1D2E2D303D245A08A1005B086F
:100C4000A00069243408303E3D243508303E3D2460
:100C50003608303E3D24592408305124A000692430
:100C600049244D24492420303D2445303D2445303D
:100C70003D242D303D243408303E3D243508303E9F
:100C80003D243608303E3D240519522E45244D247E
:100C900045248A15C6248A115908BD0008305524F8
:100CA000051D502E08004030870045244D24452462
:100CB00020303D2449303D243D303D2431303D2419
:100CC00030303D246D303D2441303D241224051A3E
:100CD000532E8030870045244D24452420303D2468
:100CE00049303D243D303D2432303D2420303D24E8
:100CF0006D303D2441303D241C24051E822E851E6E
:100D0000532E692E4030870045244D244524203041
:100D10003D2473303D2465303D246B303D2431301B
:100D20003D2430303D246D303D2441303D241C2491
:100D30005030870045244D24452420303D24733015
:100D40003D2465303D246B303D2420303D2430303F
:100D50003D246D303D2441303D241C24851E692EE8
:040D6000822E0800D7
:100E0000820700340E341134113411340A341B3487
:100E10000034003400341234123412341E341134CD
:100E2000103400340E341F341F341F341F341F3469
:100E3000003400340E3411341F341F341F341F3477
:100E4000003400340E34113411341F341F341F3475
:100E5000003400340E341134113411341F341F3473
:100E6000003400340E3411341134113411341F3471
:020E700000344C
:101000008617EB01EC01831607309F0083128701DE
:10101000871507158714B226C126B726C126B22622
:10102000203080265630802647308026413080266A
:101030003E308026B7263630802634308026303049
:1010400080262A3080263430802638308026303082
:101050008026F624803086004B2186151D30C20084
:10106000EF30C300C400EC0F3E28EB0A32306B02B5
:10107000031933214C214B21000041284B214C21E5
:101080004C2186114B218615502100000000C20B17
:101090004128C03086004B21861550210A30C500FA
:1010A00000000000000086114B218615CF3086001D
:1010B0000000CB3086000000CE3086000000CA3031
:1010C00086000000CD3086000000C9308600000098
:1010D000CC3086000000C8308600C30B53280000C7
:1010E00086114B218615CF3086000000CB3086005C
:1010F0000000CE3086000000CA3086000000CD30EF
:1011000086000000C93086000000CC308600000058
:10111000C8308600C40B7028000086114B2186154C
:101120005021851EA128C50B8D28000086110000C6
:101130000000000086155021051D56290000803052
:101140002B288617EB01EC01B226C126B726C12653
:10115000B226203080265630802647308026413007
:101160008026B726313080263230802638308026DF
:10117000303080262A30802631308026303080265C
:101180003230802634308026F62480308600463087
:10119000C2008615EC0FD228EB0A32306B0203191D
:1011A0003321D5284B2100000000F030C300C400DB
:1011B00086110000000086154C2100000000C20BC3
:1011C000D828C03086000000000086154C210A3067
:1011D000C5000000C830860086110000CA308615A0
:1011E00086004B2100000000C830C30BEB28000034
:1011F000860086110000C930861586004B21F0302C
:10120000C300C830C40BF828000086008611000017
:10121000CC30861586004B21F030C400C830C30B9B
:1012200005290000860086110000C9308615860059
:101230004B2100000000C830C40B122900008600BA
:1012400086110000000086154C21851E0028C50B64
:101250002029000086110000000086154C21051D84
:1012600056298030C628B226C126B726C126B22606
:1012700020308026503080265730802652308026FD
:101280005F3080266F30802666308026663080266C
:10129000861348290800080000000000000008002C
:1012A0000530BE00BE0B522900000800EB01EC0126
:1012B0008617B226C126B726C126B2262030802640
:1012C0004C3080268224F624D701831607309F00F5
:1012D0000130870083128B130630900010108715A1
:1012E00007158710EC0F7929EB0A03306B020319FD
:1012F000332105197C29222B851D7F29542A0A2494
:101300000130210203188F298330200203188F290E
:10131000B226C126B726C126B2268D247229EB013A
:10132000EC012108A5002008A4002325A701A6019F
:101330000330A500E830A4003A252108C7002008A2
:10134000C600051AA729F624051AA72920240F305C
:10135000A3001930A2000D30A1002030A000A70189
:10136000A60124305F24A50025305F24A4003A257F
:10137000A701A6010330A500E830A4002325A7019A
:10138000A6014708A5004608A4003A252108C9007F
:101390002008C8004B1CD229A701A601A501643072
:1013A000A4002325A701A60128305F24A500293029
:1013B0005F24A400B226C126B726C126B2264C302F
:1013C0008026783080262030802616252C1CEA299D
:1013D0002D308026CB2501302D0203183A2A01300A
:1013E0002E0203183A2A01302F020318222A013054
:1013F00030020318252A013031020318282A01304F
:1014000032020318082A0130330203180B2A0E2A6D
:101410003208303E80263308303E80263408303E85
:1014200080262C3080263508303E80263608303E17
:10143000802620308026753080266B30802648300C
:10144000802672292F08303E80263008303E8026C4
:101450003108303E80262E3080263208303E8026ED
:101460003308303E8026203080266D30802648307C
:10147000802672292D08303E80262E08303E802698
:101480002C3080262F08303E80263008303E8026C3
:1014900031082030802648308026653080266E3026
:1014A0008026203080267229EB01EC018617B226B7
:1014B000C126B726C126B22620308026433080269A
:1014C0008224F624D701EC0F6A2AEB0A03306B0260
:1014D0000319332185196D2A56290519702A222BE3
:1014E0000A24023021020318802AFE302002031849
:1014F000802AB226C126B726C126B2269A24632A9C
:101500002108A5002008A4002325A701A601033077
:10151000A500E830A4003A252108A5002008A40071
:101520000F30A3001930A2000D30A1002030A00020
:101530003A25051AAC2AF624051AAC2AB226AD249F
:10154000B726C1262108BD002C306A242008BD0022
:101550002D306A24F624BC264B1CB42AA701A60110
:10156000A5016430A40023252C305F24A5002D3074
:101570005F24A400A701A601B226C126B726C12672
:10158000B2264330802678308026203080261625EB
:101590002C1CCC2A2D308026CB2501302F0203189D
:1015A0000F2B013030020318FA2A013031020318E0
:1015B000FD2A013032020318E22A013033020318F7
:1015C000E52AE82A3208303E80263308303E80265D
:1015D0003408303E80263508303E80262C30802668
:1015E0003608303E802620308026703080264630F7
:1015F0008026632A3008303E80263108303E80261F
:101600003208303E80262E3080263308303E802639
:10161000203080266E30802646308026632A2F08B0
:10162000303E80262C3080263008303E802631081F
:10163000303E802632082030802602308026463018
:101640008026632AEB01EC018617B226C126B72655
:10165000C126B22620308026463080268224F624F9
:10166000051D302B871507118714EC0F382B3321FC
:101670000519522BB226C126B726C126B226203024
:1016800080264530802653308026523080262030F8
:1016900080263E308026F624831684309F008312F5
:1016A0008A114D286123B226C126B726C126CB2533
:1016B000B22646308026783080263E30802695231C
:1016C000352B06309000E530C1000430BD00A0018C
:1016D000A101A201A3018F018E010C10101448304A
:1016E000BE000230BF00BE0B732BBF0B732B0C1C54
:1016F0007F2BA20A0319A30A0C100000852B0000FF
:1017000000000000000000000000C10B6F2BBD0BAB
:101710006F2B000010100C1C902BA20A0319A30AB7
:101720000F08A1000E08A000080001302F020318C6
:10173000A62B013030020318AB2B01303102031805
:10174000B02B013032020318B72BBC2B82309B2602
:101750002F08303E802683309B263008303E80267E
:1017600084309B26203080263108303E802686300B
:101770009B263208303E802687309B263308303E39
:101780008026203080263408303E80263508303EC2
:1017900080263608303E802620308026483080263D
:1017A0007A308026080026309000C830C100023010
:1017B000BD00A001A101A201A3018F018E010C10A7
:1017C00010141E30BE000230BF00BE0BE52BBF0B55
:1017D000E52B0C1CF02BA20A0319A30A0C10F52B05
:1017E00000000000000000000000C10BE12BBD0B59
:1017F000E12BB330BE00BE0BFB2B0000000010102D
:101800000C1C052CA20A0319A30A0F08A1000E083C
:10181000A0000800D323013022020318162C1F3029
:1018200021020318162C0130CB001D2CCB01A7017F
:10183000A601A5010A30A4003A25A701A6010800C7
:10184000B226AD240F30A3001930A2000D30A10044
:101850002030A000A701A6014708A5004608A40063
:101860003A25A701A601A5010A30A4003A252108BE
:10187000BD0024306A242008BD0025306A24CB2511
:10188000B7264330802678308026203080263408E2
:10189000303E80263508303E80263608303E802691
:1018A00070308026463080264808BD0029306A24E2
:1018B0004908BD0028306A24F624BC260800031716
:1018C00083128D0083168C130C1483120C080313DF
:1018D00083120800031783168C186C2C83128D005A
:1018E000031383123D0803178C0083168C130C1509
:1018F0008B1355308D00AA308D008C140C110313FE
:1019000083120800203080264D30802665308026E6
:1019100074308026723080260800203080264C30BB
:101920008026783080262D3080262D3080262D3060
:10193000802608002030802643308026783080269C
:101940002030802645308026523080265230802636
:101950004F308026523080260800203080264330C9
:101960008026613080266C30802669308026623087
:10197000802672308026613080267430802669305F
:1019800080266F3080266E3080260800203080262A
:101990005330802661308026763080266530802660
:1019A00020308026453080264530802650308026E5
:1019B000523080264F3080264D30802608009730E8
:1019C000BE000330BF00BE0BE32CBF0BE32C0800AE
:1019D000AC30BE001330BF000630C000BE0BEE2C92
:1019E000BF0BEE2CC00BEE2C000008005430BE00E4
:1019F0008A30BF000330C000BE0BFC2CBF0BFC2C98
:101A0000C00BFC2C00000800A401A501A601A70141
:101A10000800A001A101A201A301A401A501A60142
:101A2000A701A801A901AA01AB0108003D260318DE
:101A3000080023082706B7000626031027082306F8
:101A4000B71F803E0800B7012726031C3A2603185B
:101A50000800152622261F30B8004D262B0D03182E
:101A60000626031C230D03180800B80B2D2D37186C
:101A70002A260800B7012408250426042704003C70
:101A8000031C2726031C3A2603180800A801A901F5
:101A9000AA01AB014D261F30B8004D2627082B02A6
:101AA000031D5C2D26082A02031D5C2D2508290232
:101AB000031D5C2D24082802031C6E2D2408A80297
:101AC0002508031C250FA9022608031C260FAA02BD
:101AD0002708031C270FAB0203102014B80B4D2D51
:101AE00037182A260800B701272603105126270891
:101AF0002B02031D852D26082A02031D5C2D2508B7
:101B00002902031D852D24082802031C902DA00FF7
:101B1000902DA10F902DA20F902DA30A031908005C
:101B200037182A260800230D0318080015261E263C
:101B30001030B800A80DA90DAA0DAB0DA40DA50D70
:101B4000A60DA80DA90DAA0DAB0DA40DA50DA60DF2
:101B50000314A00DA10DA20D22082602031DB62D0F
:101B600021082502031DB62D20082402031CC32DC5
:101B70002008A4022108031C210FA5022208031C2F
:101B8000220FA602A0142010B80B9A2D0310A20C4D
:101B9000A10CA00C0800B701272603180800562640
:101BA0002030B800A00DA10DA20DA30D3630840089
:101BB0000A30B900800D0A30000203188000840347
:101BC000B90BDA2DB80BD22D37182C1403100800DE
:101BD000B7002030B8002C3084003708B9000A3034
:101BE0000310840A03188007800CB90BF12DA30C95
:101BF000A20CA10CA00CB80BEB2D0008FF3E031C9F
:101C0000230D031808002C182A2608002408A00712
:101C100025080318250FA10726080318260FA20779
:101C200027080318270FA30708002008A800210889
:101C3000A9002208AA002308AB000800A401A501FE
:101C4000A601A701A001A101A201A3010800230D83
:101C5000031C080023088039A009A109A209A309CF
:101C6000A00F372EA10F372EA20F372EA30AB70AC7
:101C700023070800270D031C080027088039A40942
:101C8000A509A609A709A40F4A2EA50F4A2EA60F3B
:101C90004A2EA70AB70A27070800A00DA10DA20D1A
:101CA000A30DA80DA90DAA0DAB0D0800AC01AD0147
:101CB000AE01AF01B001B101B201B301B401B50190
:101CC000B6010800C826C826C8260330C200860010
:101CD00086160000000000008612C826C20B682E7F
:101CE0000230860086160000000000008612860181
:101CF000D12628309B260C309B2606309B260800D8
:101D0000BD003D0E0F3910388604E0388605861672
:101D100000000000000086123D080F3910388604CC
:101D2000E0388605861600000000000086121F308D
:101D30008604D1260800BD003D0E0F398604E03828
:101D40008605861600000000000086123D080F3947
:101D50008604E03886058616000000000000861222
:101D6000D126080080309B260C309B260800C0300E
:101D70009B260C309B26080001309B260C309B26AE
:101D800008001030C20020308026C20BC32E08008D
:101D90002F30BE000630BF00BE0BCC2EBF0BCC2EAA
:0C1DA00008004130BE00BE0BD32E08002E
:02400E00713F00
:104200007F0000007F0000007F0000000000000031
:1042100003000000000000007F000000000000001C
:1042200064000000000000006400000000000000C6
:10423000000000000000000000000000000000007E
:10424000000000000000000002008A0000000000E2
:1042500027001000000000001900640000000000AA
:00000001FF
